:10740000E0E0F0E0859194910196089520E82093C2
:1074100061001092610081E085BF82E085BF81EF4D
:1074200085B987EE84B984E08DB984E48EB910BA49
:1074300080EF81BB80E68BB980EF8AB980E58CBD97
:1074400081E08DBD089580EE8BB98BEA55D0109206
:1074500089008AEF8093880082E080936F0083E048
:1074600080938100E7E0F1E05CD0E331E9F7A5E249
:10747000B4E0E3E1F1E003E010E101900D921A9530
:10748000E1F7A059BF4F0A95B9F753D081E0809337
:10749000D7008AE482BF1092D8001092E2001092C6
:1074A000DA001092E10080E808D019BC1EBA1092F0
:1074B000E0006CD489E058D481E98093D800089525
:1074C000F201F999FECFF2BDE1BD0895F9DFF89A16
:1074D00080B508C0F5DF1FBA80BD0FB6F894FA9AE0
:1074E000F99A0FBE31962F01089590E81BD08D9325
:1074F0009A95E1F7089586E008D010C083E005D0A2
:107500008F2F10D08E2F0ED080E05E9A72980AC016
:1075100005D085E0FADF06D080FDFDCF729A5E9837
:10752000089581918EBD8DB5000087FFFCCF8EB58B
:107530000895EDEEF2E090EB5C98892FF3DF80E1A7
:10754000F1DF5C9AEEDF8DEE8E278F77D9F793957A
:10755000983B91F70895EBEDF1E0819190810196D0
:1075600090838293092E0AF400940091D90106FBBE
:107570005EF00096929111F493959083000C08169A
:1075800020F42E9A2F9A2D9A0895937009F42E982C
:10759000913009F42F98923009F42D980895E2ED76
:1075A000F1E097819923EAF08FB18095807F669B07
:1075B00088601C9B84609581891310C096819923F3
:1075C00081F49381891306C09481992396E959F037
:1075D00080E00AC083839095892304C085839AE064
:1075E000968380E09FEF9483828308958091D901F0
:1075F00086FFC7DF22243324E2EDF1E010861186F6
:107600001286EDEEF1E08091D40187FD1BC084FD70
:1076100032C082FF0895C685CC23E1F3F894289800
:107620000088F785E02D6ADFE0E0F0E0ADEEB1E044
:107630005CDFADEEB1E03ED3E058FF4FCA95B1F745
:107640006DDFC9C18301282D6090F6017090F501AE
:1076500046D019F48823C1F70895380188243FD013
:10766000E1F58091F401821709F483016090F8013B
:107670007090F701F4CF6090F8017090F7012FD06F
:1076800081F48823C1F708959FEF85FD08C086FD2A
:1076900005C083FF0895B4DEE9F39DC191E097FB37
:1076A000890E662477248301222719D0B1F4882318
:1076B00089F38091F40136F0881650F4821730F087
:1076C000213003C0881520F4281710F48301282FD7
:1076D0006090F8017090F701E8CF3801822EF30135
:1076E0000DDFADEEB1E001DFCDEED1E0E0E0F1E0A5
:1076F00097E009908191081621F49A95D1F70880B6
:1077000080100CCFC9E0F1DECA95E9F707DF11DF81
:047710008827089529
:1077140041524455424F59D5F08D14A1C881CFD957
:10772400F1AF000000FFFFCFCFFFFFFFFFCFCFFF80
:10773400FF0000FE067E7E06FE46565616FE0656E0
:10774400461EFE3F61E9E3FFE3EBE3FFE3EBE3FF08
:10775400E16B3F12011001020000084123360001D1
:10776400000201000109023E000201008032090406
:107774000000010202010005240010010424020497
:107784000524060001070582030800FF090401001F
:10779400020A000000070504021000010705830225
:1077A40010000104030904220341007200640075FF
:1077B4000069006E006F0020004C0065006F006ED1
:1077C400006100720064006F0018034100720064DD
:1077D40000750069006E006F0020004C004C0043EF
:0277E4000000A3
:1078000011241FBE8DEF9AE09EBF8DBF04B714BE3A
:1078100088E18093600010926000409100085091D0
:1078200001086F917F91A6C00F928F939F931F9233
:107830000FB60F9211244F936F938091DA0080FF5F
:107840004CC038C00F920FB68F939F93EF93FF9366
:1078500088278093850080938400E2EDF1E0978192
:10786000907261F490818917980B908309F45D9A66
:1078700091818917980B918309F4289A96819150E8
:1078800008F096839481915008F09483881639F417
:107890007C9B05C0B5DD19F0C10101961C01FF916B
:1078A000EF915CC080E189BD82E189BD09B400FE31
:1078B000FDCF08958091D80080FF0FC08091DA003D
:1078C0008E7F8093DA008091D90080FF04C0EADFC8
:1078D00081E08EBB02C019BC1EBA8091E10080FF1E
:1078E0000BC03CD280FF08C03CD28091D80080629F
:1078F000E4DD19BC85E08EBB8091E10084FF1AC0F5
:107900002DD284FF17C0CEDF8091D8008F7DD5DDCA
:107910008FEE2AD023D28F7E816026D28091DD0126
:10792000882331F48091E30087FD02C081E001C02B
:1079300084E08EBB8091E10083FF0CC00FD283FFF7
:1079400009C087EF11D082E08EBB1092DD010BD011
:1079500008D21CD26F914F910F901F909F918F91E1
:107960000FBE0F9018958EEF0090E1000822009254
:10797000E10008954BDDA0E0B1E0E4E1F7E7059018
:107980000D92A13DE1F71D92BB30E9F701FD0FC05B
:1079900000FF03C07C9B0BC008C003FF08C06757F3
:1079A000774729F04757574711F02ADDA1F44BDDFF
:1079B000222433243101882492DE789447D00AD3DC
:1079C000EEDD62DE811411F011DEF8CFC4DDC101FD
:1079D000805B964398F3F89489EB8EDD81E0809389
:1079E000E00010926F0010928100109285001092BA
:1079F000840081E085BF15BEC4DD5D9A289A0C9491
:107A00000000A7D107C054D102C0E1D239F0A3D100
:107A100082FFFBCF85FFF7CF8091F1000895082EFC
:107A200083E098D185FD07C08DD102C0D0D269F026
:107A300092D180FFFBCF0092F1008091D90185FBAC
:107A400026F05D9884E68093D201089582D182FF6A
:107A50004AC18091D90185FB26F0289884E680935D
:107A6000D301CFDF182F853431F48CEB94E31C0164
:107A700027DD8DE008C1843511F4C3DFFACF8C34E3
:107A8000C1F38035B1F3843721F484E4C8DF80E0AA
:107A9000FAC0813611F489E5F6C0813429F4B1DFEA
:107AA000582EAFDF482EE5CF803711F483E5EBC0C9
:107AB000833539F4C0E0D1E08991B1DFC730E1F717
:107AC000E3C0863521F481E3AADF84E3DCC0863796
:107AD00061F481E3669B8E5F1C9B8F5FA0DF8FB19B
:107AE000809582958F708F5BCEC08837A9F489DF2F
:107AF0008093D901289A84FD28985D9A83FD5D982A
:107B00002E9A81FD2E982F9A82FD2F982D9A80FD16
:107B10002D9887FD8824ADCF8A3649F48FE9F5DCAE
:107B2000C3E000DD7CDFCA95E1F7F8DCADC0833748
:107B300031F487E874DF85E972DF8EE1A4C0853611
:107B400039F4E0E8F3E7C7D0E058F040E0F791CF30
:107B5000823631F489E563DF80E061DF80E893C03D
:107B6000823419F0873609F07AC02224332449DFA1
:107B7000D82F47DFC82F45DF082F8354843008F003
:107B800081C0063411F4440C551CF20110926F00B0
:107B90001736A1F4033471F483E0B1DCC3DC3FDFBA
:107BA0002197E1F7BBDC08C0063411F4859101C0D0
:107BB0008DDC35DF2197C2F72F0149C00334A1F4D2
:107BC0008E2F8F7021F497DC80E299DCA1DC93DCAE
:107BD00082E095DC16DFA6DCCA95E1F799DC3196E8
:107BE000DA9571F72F0131C00634F1F49F01F437B3
:107BF000D8F471D019C005DF063461F4C0FB46F03B
:107C0000F43728F4182E81E087BFE89511243296C6
:107C1000082E0AC0043439F4DF01B370A351BD4FFC
:107C20008D93319601C056DC21972AF7043431F444
:107C30002F01F370FE2B49F47CDC07C0063429F4D5
:107C40002F01F901F43708F444D08DE0E8DE063462
:107C500011F45694479482E080936F0015C08237E8
:107C6000E1E049F08634E0E031F08E34E3E019F0F1
:107C7000813531F4E2E0F0E089E087BF849103C010
:107C80008B3111F08FE3CBDE83E0B1D15BD095FF78
:107C900003C009C09CD139F15ED080FFFBCF52D028
:107CA00002C095D101F157D080FFFBCF84E09FD176
:107CB0008BE749C0F437B8F40ED090E40D901D90D6
:107CC00081E087BFE89532969A95C1F71124E05874
:107CD000F04085E001C083E001D081E187BFE895F5
:107CE00007B600FCFDCF08959091E5018091E60173
:107CF000913231F0913A61F5813251F538D087C037
:107D0000803231F534D063D1E9F08530D9F023D019
:107D100083FD18C082FFF7CF04C07EDE81936150DF
:107D200031F09091F3008091F200892BB1F7C0DF20
:107D3000611549F704C04BD129F0853019F00BD0FB
:107D400080FFF9CF8EE79091E80089238093E800C7
:107D5000089584E04CD18091E80008958091E2007C
:107D60000895FCDF8E7F80618093E20008952DD11D
:107D7000EEEDF1E067E0089582E061EC09D083E088
:107D800061E802D084E060E842E103C080E060E0A6
:107D900042E02DD181E007D01092ED006093EC001D
:107DA0004093ED0008959091EB00892B8093EB00B8
:107DB000089560E0923039F0933041F0913099F4B9
:107DC000E3E462E110C0E5E56EE30DC0813018F434
:107DD000E3E964E008C019F4E7E962E204C0823034
:107DE00011F4E9EB68E1F1E008958091E501882361
:107DF0004CF402C0ECD051F0AEDF82FFFBCF58CF85
:107E0000E6D021F0A8DF80FFFBCF9CDF08954091F2
:107E1000EB015091EC014617510510F490E028C099
:107E2000611511F0462FFACF8DDF40E0F7CFCFD0AC
:107E300059F1853049F18FDF83FD3ACF8CDF82FD28
:107E400020C080FF15C03091F3002091F20005C0E2
:107E500081918093F10041502F5F411519F0283036
:107E60003105B0F350E02830310509F451E06ADF04
:107E70004115E9F65523D9F604C0A9D029F085307B
:107E800019F069DF82FFF9CF13CFE5EEF1E0C4DD31
:107E90008193ED3EE1F728DF5EDF83FF91C08091A3
:107EA000E5019091E601913009F170F09330F1F025
:107EB000953009F444C0963009F456C0983009F45E
:107EC00060C0993059F767C0823841F78091E90165
:107ED0008DD02091EB001092E90077D02295269565
:107EE00021702093F1001092F10052C0882311F00C
:107EF0008230A1F68F71823089F68091E701882364
:107F0000D1F42091E901277049F22093E900809192
:107F1000EB0080FF10C0933011F480E20BC080E1D1
:107F200042DF81E0880F2A95E9F78093EA001092FA
:107F3000EA0088E038DF1092E90047D02AC08823A1
:107F400091F41091E70110680FB7F8943ED04DDF1F
:107F500002DF80FFFDCF1093E300103883E009F4C7
:107F600082E08EBB0FBF2CC08058823048F58091D4
:107F7000E7019091E8011DDF603011F126D047DF65
:107F80001FC08038E9F421D08091DD018093F10099
:107F9000D9DE2BDF15C0882399F49091E701923048
:107FA00078F49093DD0111D020DF8091DD018823EA
:107FB00021F48091E30091E087FD94E09EBBDCDE3C
:107FC000CADE83FF089580E2EEDE87EFBCCE8EB37B
:107FD00088230895FCDF69F08091E9008F93109267
:107FE000E900B9DE83FF01C050DF8F918770809375
:047FF000E900089507
:047FFC005BCEFBDC81
:040000030000740085
:00000001FF
